:10000000130A4903890128006803890389016803E9
:10001000A801280369030008010C210040008101A8
:1000200043070E0A0008D50C0200FC0C0600210C48
:1000300029000604260406022C006C07280A4C0638
:10004000220A250A060526051B0A060426041B0AA1
:100050000604260506022C008C073D0A6C063A0AA7
:100060000C09260406022C008C073D0A6C061B0AAC
:100070000C09280A260406041B0A010909022B00A0
:10008000070C2A0026050C0906022C008C06280AFB
:100090006C063A0A26040C0906022C008C06280A73
:1000A0006C061B0AEA02420AEB02400A0605000C33
:1000B0002B00070C2A0026050C0906022C008C06D2
:1000C000280A6C063A0A26040C0906022C008C0643
:1000D000280A6C063A0AEA025B0AEB02590A01098D
:1000E00009022B00150C2A0026050C0906022C001B
:1000F0008C06280A6C063A0A26040C0906022C0013
:100100008C06280A6C063A0AEA02740AEB02720AA2
:100110000604260506022C006C063A0A8C06280AFC
:100120000C09260406022C006C063A0A8C06280AE2
:040130000C09890A23
:00000001FF
